:100000000C9498020C9400290C94D0020C94D00209
:100010000C94D0020C94D0020C94D0020C94D00218
:100020000C94D0020C94D0020C94961F0C94D21E07
:100030000C9453190C94D0020C94D0020C94D0025E
:100040000C94D0020C94D0020C94D0020C94D002E8
:100050000C94D0020C9406190C94D0020C94D0028B
:100060000C94D0020C94D0020C94D0020C94D002C8
:100070000C94D0020C94D0020C94D0020C94D002B8
:100080000C94D0020C94D0020C94D0020C94D002A8
:100090000C94D0020C94D0020C94D0020C94D00298
:1000A0000C94D0020C94D0020C94D002DB06DB0638
:1000B0000D070D077F072709270927099B077908DF
:1000C0008A088A08EB1C121DAA1E121DAA1E5A1DA0
:1000D0007D1DAA1E6C1E7F1E00047F3F1F6432140C
:1000E000643214783C1E1E140A0522232526282972
:1000F0002A2C2D2F3032333536383A3B3D3E4042A4
:10010000434547494A4C4E5051535557595A5C5EE6
:100110006062646668696B6D6F71737577797B7DFA
:100120007F81838587898A8C8E90929496989A9CF9
:100130009E9FA1A3A5A7A8AAACAEAFB1B3B4B6B811
:10014000B9BBBCBEBFC1C2C3C5C6C7C9CACBCCCD73
:10015000CED0D1D2D2D3D4D5D6D7D7D8D9D9DADA4E
:10016000DBDBDBDCDCDCDCDCDDDDDDDDDCDCDCDCCE
:10017000DCDBDBDBDADAD9D9D8D7D7D6D5D4D3D202
:10018000D2D1D0CECDCCCBCAC9C7C6C5C3C2C1BFE0
:10019000BEBCBBB9B8B6B4B3B1AFAEACAAA8A7A544
:1001A000A3A19F9E9C9A98969492908E8C8A898700
:1001B0008583817F7D7B79777573716F6D6B6968DE
:1001C000666462605E5C5A5957555351504E4C4AB2
:1001D0004947454342403E3D3B3A3836353332305D
:1001E0002F2D2C2A29282625232205010980A1014B
:1001F000850319012AB700150126B700950175106E
:100200008100C0050C0901A101850419012AA00281
:10021000150126A002950175108100C0050109068F
:10022000A101050719E029E71500250195087501C9
:1002300081029501750881010507190029FF150044
:1002400026FF009506750881000508190129059506
:100250000575019102950175039101C009023B00EA
:10026000020100A0FA0904000001030101000921B4
:100270001101000122400007058103080001090463
:1002800001000103000000092111010001223200D8
:10029000070582032000011201000200000008107F
:1002A000CB58120001010200011C0346006F006CD4
:1002B0000064004B00420020005200650076002ED2
:1002C000002000310000000E034B00650065006255
:1002D0000069006F00000004030904A8002900352C
:1002E000001E001F002000210022004A0000002BF9
:1002F0000014001A000800150017004D0000003916
:100300000004001600070009000A004B000000E18D
:10031000001D001B000600190005004E000000E053
:1003200000E300E20001512C002C002300240025F2
:1003300000260027002D002E002A001C0018000CAB
:1003400000120013002F00300031000B000D000ED2
:10035000000F0033003400000028001100100036A8
:100360000037003800E500000001512C002C00008F
:1003700000E600E70076000000E400A800005C0151
:1003800000C75CC65C010001000100C15C00000107
:1003900000C95CC85C010001000100C45C000001F0
:1003A00000CB5CCA5C010001000100A90000000153
:1003B0000001000100010001000100AA000000018D
:1003C0000001000100010001000100010001000125
:1003D0000001000100010001004C00010024002583
:1003E000002600010001000100010001002100229F
:1003F000002300010001000000010001001E001F99
:1004000000200001000100000001000100270000A1
:1004100000010001000100000001000001010101D4
:1004200001010101010202020202020202020303AF
:10043000030303030303040404040404040505057F
:100440000505060606060607070707070808080841
:10045000090909090A0A0A0B0B0B0C0C0C0D0D0DEE
:100460000E0E0E0F0F0F1010111111121213131484
:1004700014151516161717181819191A1A1B1B1CFC
:100480001D1D1E1E1F202021222223242425262656
:10049000272829292A2B2C2D2D2E2F30313232338B
:1004A0003435363738393A3B3C3D3E3F4041424394
:1004B0004445464748494A4C4D4E4F505153545578
:1004C0005658595A5B5D5E5F616264656668696B28
:1004D0006C6D6F7072737577787A7B7D7E808283A6
:1004E0008587888A8C8E8F91939596989A9C9EA0EA
:1004F000A2A3A5A7A9ABADAFB1B3B5B7BABCBEC0F7
:10050000C2C4C6C9CBCDCFD1D4D6D8DBDDDFE2E4BF
:10051000E7E9EBEEF0F3F5F8FAFDFFFFAA7F5540AF
:10052000000102030C0D0E0F0405060708090A0B53
:1005300011241FBECFEFDAE0DEBFCDBF04B603FE4D
:1005400018C080912D0390912E03A0912F03B0919C
:1005500030038730904BA740B04B59F410922D03D5
:1005600010922E0310922F0310923003E0E0F8E374
:10057000099511E0A0E0B1E0EEE3F6E502C00590D8
:100580000D92AE3CB107D9F723E0AEECB1E001C06B
:100590001D92AD32B207E1F70E948B110C941D2B16
:1005A0000C9400001F93CF93DF93CDB7DEB767970E
:1005B0000FB6F894DEBF0FBECDBF4B8B5C8B6D8B3F
:1005C0007E8B8F8B611110922C0386E09E01235F3E
:1005D0003F4FD901E82F1D92EA95E9F795E0FE011A
:1005E0007396D90101900D929A95E1F79C894E89F5
:1005F0005F897B897D879E876F87598B488BF9013F
:10060000DE01179601900D928A95E1F7CE010796CB
:100610000E94C62181113EC086E0FE013796DE01B0
:10062000119601900D928A95E1F7FF81E8856A8520
:100630007B856115710531F0EF3F31F481E0FF3FBB
:1006400019F403C081E001C080E080FD23C0209147
:10065000F10230E0C9010196877099274091220389
:1006600050E08417950779F1F983EA837D836C83E1
:1006700096E0929FD001939FB00D1124AE50BD4FD4
:10068000FE01319601900D929A95E1F78093F10267
:100690000E94B52016E0809122039091F102891703
:1006A000F9F0189FC00111248E509D4F0E94C62161
:1006B0008823B1F08091220390E0019687709927FA
:1006C00080932203E8CF0E9452241092F1021092EC
:1006D0002203EBEEF2E086E0DF011D928A95E9F756
:1006E00067960FB6F894DEBF0FBECDBFDF91CF91F6
:1006F0001F91089581110AC0662321F060E070E027
:1007000089EA0FC060E070E08AEA0BC0813059F4DA
:10071000662321F060E070E08EE403C060E070E0EA
:100720008BE40E946E2480E008958F929F92AF9296
:10073000BF92CF92DF92EF92FF920F931F93CF93CE
:10074000DF93CDB7DEB72A970FB6F894DEBF0FBEA2
:10075000CDBFFC01D080118183819481892B39F038
:100760001F3F39F491E00FEFD01203C003C091E0B6
:1007700001C090E090FD9DC67F0185E0DE011696E8
:1007800001900D928A95E1F7F70122818E819F8178
:10079000222349F00E942B21082F682F8E819F81F0
:1007A0000E94932303C00E946723082FE12FF0E0EB
:1007B0001AE0019FE00DF11D112463E0EE0FFF1F11
:1007C0006A95E1F7ED0DF11DEE0FFF1FE552FD4FAC
:1007D00005911491F7018281882309F482C00E3BB0
:1007E000FCE51F07E1F058F40C3B3CE5130799F0DA
:1007F0000D3B9CE5190709F074C080E00DC0003C7A
:10080000ECE51E0709F45AC008F43FC0013C2CE592
:100810001207A9F066C083E00E943C1B6EC5809160
:100820008802982F96959695969549F1915E990F25
:10083000990F990F8770892B8093880214C090912B
:100840008802892F8695869586958F5F8F71977020
:10085000843008F043C0880F880F880F892B80935D
:10086000880280918802887F91E009F490E080916D
:10087000880290FB80F9809388020E94371B809148
:10088000880286958695869523C020918802822FBE
:10089000869586958695482F50E04330510554F44F
:1008A0008F5F982F990F990F990F822F8770892B3F
:1008B00080938802809188028160DDCF80918802D8
:1008C00080FF09C08E7F809388020E94371B80E0E2
:1008D0000E94841A12C50E94591B0FC5909388026A
:1008E000C0CF043F2CE5120749F406E221EE40EEAA
:1008F00064EF7CE5C7010E94DF19FFC4053F3CE5BA
:10090000130708F066C1093D9CE5190731F407E2B9
:1009100025EE45EE69ED7CE5EDCF0A3DECE51E07E1
:1009200031F408E221E045EE6AED7CE5E3CF083DD5
:10093000FCE51F0731F406E221EE41EE68ED7CE5AF
:10094000D9CF882309F47AC110928B0204303DE597
:10095000130758F40B3F8CE5180780F4C801825048
:100960009C45449708F054C109C002369DE519071B
:1009700029F0063AEDE51E0709F04AC10E94350E3E
:1009800090932602809325020131FCE51F0709F4AC
:10099000C6C008F042C009303CE5130709F49BC00B
:1009A00000F505309CE5190709F485C078F403309B
:1009B000FCE51F0709F478C008F07AC002301C4536
:1009C00009F0F7C0809125028160F1C007308CE505
:1009D000180709F478C008F07AC080912502806178
:1009E000E6C00D30ECE51E0709F487C058F40B3063
:1009F0002CE5120709F479C008F07BC0809125022C
:100A000088606FC00F308CE5180709F480C008F0CB
:100A100082C080912502877FCAC00E3FECE51E0789
:100A200009F471C000F505312CE5120709F485C001
:100A300068F403318CE5180709F475C008F095C017
:100A40000E945224809125028F77B1C00C3FECE5C3
:100A50001E07A9F108F054C00B3F1C4509F0A9C0BE
:100A60008091260240C002303DE5130709F489C099
:100A700058F401159DE5190709F45AC008F069C03A
:100A80008091260282602FC00236FDE51F0709F41F
:100A90007EC0063A2DE5120709F483C003301D45D8
:100AA00009F087C060E06EC08091250282607FC03F
:100AB0008091250216C080912502886078C08091BF
:100AC000260282604FC080912502806270C08091B2
:100AD000250280646CC00E945224809125028068A7
:100AE00066C0846064C081603DC0809125028E7FB5
:100AF0005EC0809125028D7F5AC08091250216C06C
:100B00008091260218C0809126028D7F2BC0809193
:100B100025028F7E4CC0809125028F7D48C0809138
:100B200025028F7B44C080912502877F8B7F3FC049
:100B3000809126028D7F8E7F15C08091250282FBD9
:100B4000222720F991E0922790FB82F990FB83F90C
:100B50002EC080912602982F909591708E7F892BC0
:100B600090FB81F98093260224C00E945224809138
:100B7000250287FB222720F991E0922790FB87F935
:100B800016C061E08EE090E00E94352A12C080918C
:100B9000250284FB222720F991E0922790FB84F91B
:100BA00006C080912502982F909590FB80F9809344
:100BB0002502609125021091260284E090E00E94B7
:100BC000352A612F82E290E00E94352A0E94522449
:100BD00094C3063F2CE5120731F406E221EE42EE03
:100BE00066EF7CE587CE063F3CE5130730F407E26D
:100BF00025EE44EE65EF7CE57DCE073F9CE51907C9
:100C000009F09FCE07E225EE46EE67EF7CE572CE57
:100C10000631ECE51E0721F58091D1018A7A91E039
:100C200009F490E09093D001882311F065E301C0AE
:100C300069E281EB92E00E9489190FC00631FCE560
:100C40001F0709F040C08091D001882309F478C3C0
:100C500065E381EB92E00E947C190E946D204DC3F8
:100C60000B35FDE51F0749F158F401153CE5130765
:100C7000B1F00F3D1C4509F042C00E94460E3DC335
:100C80000C359DE51907D9F00D351D45C1F580914D
:100C9000260282FB882780F991E0892711C00E94F3
:100CA0005224FFEF04E31CE0F15000401040E1F754
:100CB00000C000000E94E21820C381E001C080E073
:100CC0000E940A241CC08091D10182720D3C9CE5D7
:100CD000190709F4CEC308F0F9C2073CFCE51F0769
:100CE00009F4B3C308F03CC3043C3CE5130709F422
:100CF000A2C308F027C3033C1C4509F472C3F701E3
:100D0000828100811181882349F0C8010E942B2132
:100D1000D82E682FC8010E94932304C0C8010E94E6
:100D20006723D82EE12FF0E01AE0D19EE00DF11DEF
:100D3000112433E0EE0FFF1F3A95E1F7E00FF11DAC
:100D4000EE0FFF1FE552FD4F859194910E94540CC8
:100D50008C01982EF701D280A580A2945FE0A52295
:100D6000809123038770B9F0DD20A9F0812F807F67
:100D7000803421F080E2800F883068F08091260274
:100D800082FD09C082E00E94ED23809123038770D9
:100D9000CC24C3948111C12CB12EB2942FE0B22285
:100DA0008B2D90E08C30910508F051C2FC01EA5A7D
:100DB000FF4F0C94C32A812F807F1F70882311F06E
:100DC0001295107FDD20B9F0112309F42DC280E2C5
:100DD000800F883010F0911006C08091D101182B3F
:100DE0001093D10105C080912C03182B10932C0374
:100DF0000E946D2019C2802F0E946C27112309F4D4
:100E000026C2005E083078F1992069F11095809132
:100E10002C03182310932C0329C0812F807F1F706F
:100E2000803211F01295107F992021F0F1E09F1689
:100E3000D9F149C08091260282FF1BC0DD2069F0F4
:100E4000112339F08091D101182B1093D1010E9408
:100E50006D2080E00E94C327FAC180E00E946C27C9
:100E6000112309F4F4C1812F0E94BC0E0E946D2051
:100E7000EEC1DD2081F08091D201AA2051F001E085
:100E8000A01207C0182B181709F4E1C11093D20162
:100E9000DEC1812B10C0AA2021F021E0A21609F4A6
:100EA000D6C10E94B60E27C0DD2041F035E03A15CC
:100EB00008F4CDC1812F0E946424C9C184E08A1541
:100EC00008F4C5C118C0DD2049F0AA2099F3F70144
:100ED000858180FFA9C18F708583ECCFAA2059F04E
:100EE000093309F0B1C1FFEF17EE23E0F1501040D4
:100EF0002040E1F7A7C1812F0E945D24A8C1812F66
:100F000086958695837019F0813059F0A0C1DD2057
:100F100019F0C801937002C080E090E00E94B919F6
:100F20009CC1DD2019F0C801937002C080E090E000
:100F30000E94A31992C1812F837009F069C0D1105A
:100F40008AC1902F929596959770990F990F802F3F
:100F50008F70882E912CA12CB12C092E04C0880CE6
:100F6000991CAA1CBB1C0A94D2F704FF12C04FE0C4
:100F700050E060E070E004C0440F551F661F771F0B
:100F80009A95D2F7DB01CA0180959095A095B0950E
:100F900003C080E090E0DC0116951695412F437068
:100FA000423019F1C8F40091D3011091D40120917D
:100FB000D5013091D601413059F088299929AA29C3
:100FC000BB29BC01CD0160237123822393230AC076
:100FD000802A912AA22AB32ABC01CD016829792945
:100FE0008A299B290E94482436C188299929AA293F
:100FF000BB290091D3011091D4012091D5013091EA
:10100000D601BC01CD016027712782279327EACF43
:10101000DD2019F0812F817001C08695882309F4A5
:101020001AC1902F929596959770990F990F802FCE
:101030008F70882E912CA12CB12C092E04C0880C05
:10104000991CAA1CBB1C0A94D2F704FF12C04FE0E3
:1010500050E060E070E004C0440F551F661F771F2A
:101060009A95D2F7DB01CA0180959095A095B0952D
:1010700003C080E090E0DC0116951695412F437087
:101080004230D9F068F5009121021091220220919E
:10109000230230912402413059F088299929AA2944
:1010A000BB29BC01CD0160237123822393231EC081
:1010B000802A912AA22AB32A13C088299929AA2909
:1010C000BB2900912102109122022091230230912C
:1010D0002402BC01CD01602771278227932706C017
:1010E000BC01CD01682979298A299B290E94BE2348
:1010F000B2C01F70DD2039F0812F0E942724802F7D
:101100000E946424A8C0802F0E945D24812F0E9429
:10111000C823A1C0802F32EF931609F443C03915BC
:1011200038F090EF991659F0E1EF9E16B1F177C0C3
:10113000F3EF9F16F1F124EF921659F170C0DD2004
:1011400019F134E03A1508F482C01F7181E090E093
:10115000A0E0B0E0AC01BD0104C0440F551F661F04
:10116000771F1A95D2F78091210290912202A091C7
:101170002302B09124028A019B01082719272A27FC
:101180003B27C901B80129C025E02A1508F45FC032
:10119000DCCF8091260282FF23C0DD2029F0812F41
:1011A0008F7130C0DD20D9F3812F8F710E94C82349
:1011B0004EC0DD2079F01F7181E090E0A0E0B0E04A
:1011C000BC01CD0104C0660F771F881F991F1A95B7
:1011D000D2F703C060E070E0CB010E94BE2337C0AD
:1011E000DD2099F01F71812F0E9427248091260213
:1011F00082FD07C038E0139FC001112483608093F3
:101200002303812F0E94272422C081E00E94ED2326
:1012100081E08A15E0F482E00E94ED2318C0DD2011
:1012200029F0AA2009F4BBCF802F14CEAA2009F4FC
:10123000BBCF893349F49FEFE7EEF3E09150E040F4
:10124000F040E1F700C00000802F0E946C2788EF7B
:101250008B0D843010F40E94CF19CC20A9F080911E
:10126000230380FD11C0F701128285958595859530
:101270000E942724C7010E9495038091230385952E
:10128000859585950E94C82385E0F701DE011196BA
:1012900001900D928A95E1F789819A810E946723D6
:1012A000EA81F0E00AE0809FE00DF11D112483E067
:1012B000EE0FFF1F8A95E1F78981E80FF11DEE0F10
:1012C000FF1FE552FD4F85919491F3C0023D8CE5DF
:1012D000180709F4DEC008F465C0053D8CE5180761
:1012E00009F4DDC008F471C0063D2CE5120709F4CD
:1012F000DBC00E351D4509F002CD809123038770B8
:1013000009F4D7C0F7018281882309F4D2C0809103
:10131000260282FDCEC082E02A960FB6F894DEBF88
:101320000FBECDBFDF91CF911F910F91FF90EF9036
:10133000DF90CF90BF90AF909F908F900C94ED2353
:1013400069E287CC053CFCE51F0709F479C0063C3F
:101350001C4509F0D4CC47E057E260E177E28DC04C
:101360000A3C3CE5130709F47AC070F4083CECE54C
:101370001E0709F46FC0093C1C4509F0C0CC4BEFB7
:1013800056E26FEE76E279C00B3C2CE5120709F4C9
:101390006BC00C3C1C4509F0B2CC4CE455E26DE549
:1013A00075E26BC00F3CECE51E0709F46CC008F455
:1013B00067C0003D2CE5120709F468C0013D1C45DB
:1013C00009F09DCC6EE089E06CC0033DECE51E07A2
:1013D00009F462C0043D1C4509F091CC61E088E14C
:1013E00065C08091830280FF20C08E7F809383023E
:1013F00060918302709184028091850290918602AF
:101400000E943A250E94B71B80914F028160809311
:101410004F028FEF90E7E2E081509040E040E1F72B
:1014200000C000000E94852468CF81608093830201
:1014300061E086953BC049E557E262E677E21DC070
:1014400042E657E269E577E218C040E157E267E01B
:1014500077E213C04FEE56E26BEF76E20EC047ED37
:1014600056E263EE76E209C043EE56E267ED76E2BD
:1014700004C04DE555E26CE475E20E94B11B3DCF1E
:1014800061E081E013C065E082E00BC068E086E0C7
:1014900008C064E18FE005C067E185E102C062E257
:1014A00089E10E949F1B29CF61E083E20E941927F6
:1014B00024CF2A960FB6F894DEBF0FBECDBFDF91C2
:1014C000CF911F910F91FF90EF90DF90CF90BF9041
:1014D000AF909F908F90089580E00895909125029D
:1014E00092FF0DC0282F2871283019F4877F84605F
:1014F00006C0282F2471243011F48B7F886093FF5D
:101500000DC0282F2871283119F4877E846106C008
:10151000282F2471243111F48B7E886120912602BA
:1015200020FF0DC0382F3871383019F4877F816063
:1015300006C0382F3171313011F48E7F886021FF61
:101540000DC0282F2871283119F4877E816106C0CB
:10155000282F2171213111F48E7E886194FD877EC0
:1015600008956F927F928F929F92AF92BF92CF9287
:10157000DF92EF92FF920F931F93CF93DF931F920F
:10158000CDB7DEB7C62E4A015901682E880F7708FD
:10159000C3010E94A629882309F473C0C30123E074
:1015A000880F991F2A95E1F7FC01E050FF4F438116
:1015B00050E04115510511F041E050E0FC01E050D0
:1015C000FF4F6481758161517E4FCE0101960E946B
:1015D000142BF40140815181628173812FB7F894FB
:1015E0008091930290919402A0919502B0919602FD
:1015F0002FBF841B950BA60BB70B84369105A10555
:10160000B10538F4B701C8010E946D1A9981891794
:10161000D1F10C2C000CDD08C6010E94A629782E01
:101620008823E1F0E114F104C9F0960183E0220F70
:10163000331F8A95E1F7F901E050FF4F438150E0F5
:10164000E416F50608F4A701F901E050FF4F6481A4
:10165000758161517E4FC5010E94142BB701C801ED
:101660000E946D1A91E02981281390E0D92ED7208D
:1016700089F00E943B19F401608371838283938314
:1016800009C0D12C02C0DD24D394A701B801C50143
:101690000E94142B8D2D0F90DF91CF911F910F91F0
:1016A000FF90EF90DF90CF90BF90AF909F908F9082
:1016B0007F906F900895CF92DF92EF92FF920F93F9
:1016C0001F93CF93DF9300D000D01F92CDB7DEB72A
:1016D0006B0185E0E82EF12C00EF11E09E012F5FF9
:1016E0003F4F47EE51E061E080E00E94B10A88235D
:1016F00049F095E0FE013196A2EEB1E001900D9225
:101700009A95E1F795E0E2EEF1E0D60101900D92B5
:101710009A95E1F70F900F900F900F900F90DF9137
:10172000CF911F910F91FF90EF90DF90CF90089590
:101730008F929F92AF92BF92CF92DF92EF92FF92E1
:101740000F931F93CF93DF93FB0180809180A28042
:10175000B3809FB7F894C0909302D0909402E09029
:101760009502F09096029FBFC818D908EA08FB08B6
:10177000F4E6CF16D104E104F10410F4442341F15E
:101780007B01C82F880FDD0B01151105A9F0FE01A3
:1017900083E0EE0FFF1F8A95E1F7E050FF4F818154
:1017A000928181519E4F408150E00417150708F443
:1017B000A801B9010E94142BCE010E94A6298823FA
:1017C00041F00E943B19F701608371838283938308
:1017D00081E0DF91CF911F910F91FF90EF90DF900B
:1017E000CF90BF90AF909F908F9008958091E1012E
:1017F000811118C08091D80080618093D8008AE15F
:101800008A95F1F700C08091D90080FD02C082E086
:1018100001C081E08093E101823021F40E94161F13
:101820001092A70281E09091E101913009F080E0EF
:101830000895F894E82FE295EF70F0E031A1282F99
:101840002F7081E090E001C0880F2A95EAF7982F69
:101850009095932391A392A1892B82A378940895C4
:101860000F931F930E94F60B882321F01F910F9175
:101870000C943B190E943B19009111021091120225
:101880002091130230911402600F711F821F931F69
:101890001F910F9108950E94F60B81110C94471926
:1018A0000E94300CCB010895CF93DF9382389105CD
:1018B00069F1B0F48133910509F46FC048F48932BD
:1018C000910509F465C08A32910509F46BC08AC09C
:1018D0008533910509F457C089339105B9F082C069
:1018E000833E910571F138F4803E9105B1F0823E5E
:1018F000910511F177C0863E9105B9F1873E9105BA
:10190000C9F1843E910509F06DC024C020912502E3
:1019100020FD53C021FD51C065C08091250280FD8E
:1019200046C08091260280FF48C08091250284FD38
:101930003FC183EE90E03EC18091250282FF3AC014
:10194000F4CF8091250282FD35C08091260280FD72
:1019500034C0EBCF8091260281FF35C080912502F3
:1019600084FD26C187EE90E025C18091250283FF8A
:1019700027C0F4CF8091250283FD22C080912602EA
:1019800081FD21C0EBCF8091250285FD1FC021C0C4
:101990008091250285FD1DC019C08091250286FD1C
:1019A0001BC01DC08091250286FD19C015C089E3AA
:1019B00090E000C182EE90E0FDC080EE90E0FAC0C1
:1019C00086EE90E0F7C084EE90E0F4C089E290E00B
:1019D000F1C085E390E0EEC08AE290E0EBC081E3E5
:1019E00090E0E8C0811532E5930708F069C08115E1
:1019F00041E5940728F0982F8827816F906ADAC014
:101A0000883E910568F5803E910508F0D3C0883A7C
:101A10009105B8F4853A910548F0855AE82FF0E031
:101A2000E75AFE4F808190E09064C4C081309105F8
:101A300009F4BBC008F4BCC08430910508F4B8C0F8
:101A4000B9C08F3B910508F0B3C0885AE82FF0E089
:101A5000EE0FFF1FE45AFE4F808191819464AAC06B
:101A6000811520E59207F0F09C0174E036952795EA
:101A70007A95E1F7922F9370482F437021E030E080
:101A800002C0220F331F4A95E2F73C68392B8F7052
:101A9000982F9695969540E2949FC0011124822B31
:101AA000932B88C0811530E4930718F09F70906ADB
:101AB00081C09C013A9521153F4108F47BC078C054
:101AC000EC01C11586E5D807E8F5C11525E5D20773
:101AD00048F08C2F0E946E0A8F7190E0982F882713
:101AE000906268C0C11534E5D30728F09C2F882781
:101AF000846F906A5FC0AE01437055272C2F2695E6
:101B00002695C115D34578F481E090E002C0880F96
:101B1000991F4A95E2F740E2249F90011124822BFD
:101B2000932B9C6847C081E090E002C0880F991F0A
:101B30004A95E2F740E2249F90011124822B932BD7
:101B40009A6838C0C1152AE5D207F8F4C11539E5FD
:101B5000D30790F08C2F8F700E946E0A94E0D69578
:101B6000C7959A95E1F7CF70D0E0DC2FCC27D069EC
:101B70009E01282BC9011EC0C11548E5D407C0F03D
:101B80009C2F8827806F906A15C0CE0190568115D2
:101B9000904270F48D2F8F710E946E0A282F2F7142
:101BA000CE0199279062922B05C081E090E002C09F
:101BB00080E090E0DF91CF9108950C943B19CF9293
:101BC000DF92EF92FF920F931F93CF93DF931F92B9
:101BD000CDB7DEB7EE24E394F12C06EF11E09E01C1
:101BE0002F5F3F4F4BEE51E063E082E00E94B10A6D
:101BF000C82E882379F1D09028028D2D90E09C0189
:101C00002F5B3D4F79011981F9018081181B012F4C
:101C100080E010165CF40150F70180818F5F8083B3
:101C200060E08D2D0E947A0381E0F3CF912F17FDA4
:101C300090E0191B112359F01F5FF701808181503B
:101C4000808361E08D2D0E947A0381E0F3CF8111C2
:101C50000E94DD0D8C2D0F90DF91CF911F910F9180
:101C6000FF90EF90DF90CF900895CF9384E090E0C5
:101C70000E94212AC82F82E290E00E94212A2C2F64
:101C800030E0A901582BCA01CF91089569EE7EEF8B
:101C900080E090E00E94532A60E082E090E00E94A1
:101CA000352A60E083E090E00E94352A1092D3014B
:101CB0001092D4011092D5011092D60160E084E018
:101CC00090E00E94352A60E082E290E00E94352A8E
:101CD00060E085E090E00E94352A60E086E090E0D8
:101CE0000E94352A6FEF87E090E00E94352A40E09D
:101CF00050E0BA0188E090E00E94472A60E08DE061
:101D000090E00E94352A40E050E0BA0188E190E07E
:101D10000E94472A60E087E190E00E94352A40E077
:101D200050E0BA018CE190E00E94472A60E070E048
:101D300080E290E00E94532A40E050E0BA0188E13E
:101D400090E00E94472A0E94591B83E00E943C1B9E
:101D500040E050E0BA018FE090E00E94472A40E066
:101D600050E0BA0183E190E00C94472A8091D201BF
:101D700081111092D201089580959091D10189230B
:101D80008093D10108955F926F927F928F929F927C
:101D9000AF92BF92CF92DF92EF92FF920F931F9379
:101DA000CF93DF93CDB7DEB72F970FB6F894DEBF92
:101DB0000FBECDBF9E012F5F3F4F79018AE0D90151
:101DC0001D928A95E9F70CE811E0690181E9682E16
:101DD00081E0782EAA24A394B12C29E9822E21E057
:101DE000922EF80180818F3F09F440C0F894E82FCB
:101DF000E295EF70F0E021A18F70A50102C0440FC1
:101E0000551F8A95E2F7CA01922F982B91A392A1B0
:101E10008095892382A3789400C0E1E9F1E0512CF8
:101E200031E021912F3F89F0A22FA295AF70B0E051
:101E300090968C9190E02F7002C0959587952A9589
:101E4000E2F780FD02C0832F01C080E0582A330FE3
:101E50008E169F0631F7D8018C918F3F11F00E94AA
:101E6000190CB0EABA95F1F7F60150820F5F1F4FD7
:101E7000FFEFCF1ADF0A6016710609F0B2CF4AE011
:101E800050E0B70185E192E00E94072B8C01892B7D
:101E900041F08AE0F701A5E1B2E001900D928A9548
:101EA000E1F7F09020020115110549F081E08093DF
:101EB000D9010E9447199093D8018093D70180914E
:101EC000D9018823B9F08091D7019091D8010E945F
:101ED0002C19059778F0A5E1B2E0EF2DF0E0E75D71
:101EE000FD4F8AE192E02D9121938A179B07D9F744
:101EF0001092D9010115110509F026C10E94F60BB7
:101F0000E09120029E01255F3F4F7901882309F46B
:101F10006DC085E0D9011D928A95E9F70E2F10E07A
:101F2000075D1D4F809110028A3048F44BE55BE05D
:101F3000B701C8010E94CB14882359F10AC08091CF
:101F4000DA019091DB010E942C19843F914070F7D7
:101F500032C04FED5DE0B701C8010E94CB14882369
:101F6000C1F043E351E1B701C8010E94CB148823BB
:101F700081F04CE051E1B701C8010E94CB148823E5
:101F800041F041ED50E1B701C8010E94CB1481112D
:101F9000DEC0809110028F3F19F08F5F8093100296
:101FA000809110028A3008F4D4C00E94471990939F
:101FB000DB018093DA018091E001811102C000E031
:101FC000D9C085E0F70111928A95E9F71092E001F6
:101FD000A0911F02B0E0A75DBD4F85E0FE013B96DA
:101FE00001900D928A95E1F701E0C4C0F0E0E75D51
:101FF000FD4FF89485E0A0EFB1E001900D928A9535
:10200000E1F765E070E080EF91E00E946D1A809347
:10201000EF017894F894E0914402F0E0EF5BFD4F1B
:1020200080818B878093F60161E070E0C7010E9498
:102030006D1A8093F5017894F894C090F701D090D0
:10204000F801E090F901F090FA018091DC019091A3
:10205000DD01A091DE01B091DF01C816D906EA06C4
:10206000FB06D1F0C092DC01D092DD01E092DE01EE
:10207000F092DF010E94F60B81110EC00E943B1905
:10208000C61AD70AE80AF90AC0921102D0921202BF
:10209000E0921302F09214027894F8948091FB017C
:1020A0000E94841A7894F89480910302882309F49A
:1020B00049C080FF24C09091FC018091830290FF71
:1020C00009C081608093830260E0892F86950E9419
:1020D000192715C08E7F809383020E94B71B8091C1
:1020E0004F02816080934F02FFEF20E732E0F15012
:1020F00020403040E1F700C000000E94852480911C
:10210000030281FF09C020E04091FF016091FE01C0
:102110008091FD010E9435268091030282FF09C053
:1021200080910202882319F00E94BE1B02C00E9407
:10213000B71B8091030283FF03C081E080934A02B2
:1021400010920302789416C001E010E013C01092C0
:10215000100280911F0290E045E050E0B701875DDA
:102160009D4F0E94072B21E02093E001892B09F06D
:102170002FCF25CF802F2F960FB6F894DEBF0FBE3E
:10218000CDBFDF91CF911F910F91FF90EF90DF9026
:10219000CF90BF90AF909F908F907F906F905F9007
:1021A00008950F931F93CF93DF93CDB7DEB7289792
:1021B0000FB6F894DEBF0FBECDBF85E0E3E8F2E0D6
:1021C000DE01119601900D928A95E1F780914D0202
:1021D00090914E02A0914F028E839F83A88741E089
:1021E0008885811101C040E008E010E09E012F5F6A
:1021F0003F4F6CE072E086E00E94980B81111092D4
:102200004F0228960FB6F894DEBF0FBECDBFDF9108
:10221000CF911F910F9108950F931F93CF93DF9349
:102220001F92CDB7DEB78091880280FF04C08695EB
:102230008695869501C080E0898341E09091FB01FD
:10224000981301C040E001E010E09E012F5F3F4F76
:1022500068E072E085E00E94980B0F90DF91CF91CB
:102260001F910F910895CF93DF9300D000D0CDB789
:10227000DEB7409104025091050260910602709110
:1022800007022FB7F8948091930290919402A09145
:102290009502B09196022FBF841B950BA60BB70B2E
:1022A00084369105A105B10570F10E94300CDC0166
:1022B000CB010296A11DB11D89839A83AB83BC8398
:1022C000809121019091220181519E4F40912001E6
:1022D00050E04530510510F044E050E0BE016F5F22
:1022E0007F4F0E94142B84E090E00E94A62988234F
:1022F00059F00E943B196093040270930502809389
:1023000006029093070281E00F900F900F900F90BC
:10231000DF91CF910895CF93DF93CDB7DEB72A97A2
:102320000FB6F894DEBF0FBECDBF84B7877F84BFE2
:102330000FB6F894A8958091600088618093600042
:10234000109260000FBE90E080E80FB6F894809382
:102350006100909361000FBE85B7806885BF85B727
:10236000806885BF8CE69AE09093CF018093CE0180
:102370000E94161F0E94351F8091E20084608093A6
:10238000E20078948091A7028823A1F01091E900DF
:102390001F709091EC00892F817090FD80E8182BC0
:1023A0001092E9008091E80083FD0E94051C1F70D7
:1023B0001093E90082E084BD93E095BD9AEF97BD4C
:1023C00080936E001092110210921202109213026A
:1023D0001092140287988F988FB1881F8827881FC2
:1023E0008093380180913801882321F010925301A5
:1023F00088E003C088E080935301809354010E94D9
:10240000F60B81110E94BA28809138018091380121
:10241000811102C095E001C090E09093200285E018
:10242000891B80931F020CE811E091E9E92E91E0ED
:10243000F92ED8018D918D018F3F11F00E94190C5A
:10244000E016F106B1F701E911E089E9E82E81E033
:10245000F82EF80181918F018F3F11F00E94190C25
:10246000E016F106B1F78AE0E9E2F2E0DF01282F99
:102470001D922A95E9F7E5E1F2E0DF011D928A95C8
:10248000E9F780E090E00E942F2A893E9E4F11F0EC
:102490000E94460E82E090E00E94212A809333023F
:1024A0000E94350E90932602809325020E94C30E4F
:1024B000EFE3FCE93197F1F700C000000E94C30E82
:1024C0008091290280FF08C06FEF7FEF80E090E0ED
:1024D0000E94532A0E94E21883E090E00E94212A81
:1024E000682F70E080E090E00E944824259A2D98A3
:1024F00082E88093800089E1809381008FEF9FEFD5
:1025000090938700809386000E94711B0E94711B2C
:102510008091270281113BC080E090E00E942F2A29
:10252000893E9E4F21F00E94460E0E946E2588E053
:1025300090E00E94292A6093830270938402809322
:1025400085029093860280914F02836080934F02B0
:102550006E7F71F40E946E2588E090E00E94292A27
:102560006093830270938402809385029093860225
:102570000E9427250E94B71B8091830280FF04C020
:1025800060E086950E94192781E080932702859854
:102590008D9A86988E9A8FE891E00197F1F700C0A6
:1025A00000008FB185FB882780F97E9902C090E0FA
:1025B00001C092E0892B809345029091380181E01F
:1025C000982790934402891B809328020E94F60B5F
:1025D000811102C00E94BD2889E391E090938F028F
:1025E00080938E02F8E1CF2ED12CA0E44A2EB3E3E3
:1025F000AB2EB2E0BB2E10E1512E8091A7028530A8
:1026000009F044C012E18091A702853009F038C07A
:102610008091A702843021F180E00E94841A1092F8
:1026200092020FB6F894A895C09260000FBE409237
:10263000600083B7817F846083BF83B7816083BF7D
:102640007894889583B78E7F83BF0FB6F894A8954A
:1026500080916000886180936000109260000FBEDE
:102660008091A602882309F4CECF0E94C30EE9E22E
:10267000F2E08191811179C1AE16BF06D1F7C3CFC7
:102680000E9452240E94711B0E94CF190E94C30E07
:1026900081110E943B19A9E2B2E0E4E3F2E000E01C
:1026A00010E0802E9D908191892549F1E12CFF2435
:1026B000F3949F2D9823F1F00E94F60B882399F054
:1026C000E9828A829F2081E009F480E08B830E9466
:1026D00047198160782F9D838C8349815A816B8152
:1026E0008D810E94D202F801EC5CFD4F8081F826BA
:1026F000F0821AC0E394FF0C98E0E912DACF0F5F82
:102700001F4F0A30110569F68FEF8E838F8318866D
:102710000E9447198160782F9A8789874E815F814F
:1027200068858A850E94D2020E94F60B80914E0233
:10273000882309F4BDC080914D02E0918302E695A3
:10274000E81BE0934902823059F4F0E0EA51FF4F70
:10275000E4910E2F10E0E9EEEE2EE7E1FE2E59C0D7
:10276000863059F4F0E0ED51FF4FE4910E2F10E068
:1027700079EDE72E77E1F72E4CC0893061F4E695CC
:10278000F0E0E052FF4FE4910E2F10E06EE5E62EF0
:1027900067E1F62E3EC08F3061F4E695F0E0E3523B
:1027A000FF4FE4910E2F10E059ECE52E56E1F52E87
:1027B00030C0853159F4F0E0E652FF4FE4910E2F1E
:1027C00010E043E4E42E46E1F42E23C08831A1F06A
:1027D000833249F4E8EDF0E00591149139E9E32EF4
:1027E00037E1F32E16C0843271F404EF11E021E7D3
:1027F000E22E25E1F22E0DC008E210E090EBE92E6A
:1028000095E1F92E06C000ED17E08DE0E82E85E198
:10281000F82E80914A02882361F010924A020E94A9
:102820004B0C909348028093470210924C021092F6
:102830004B020E944B0CE0914702F09148029C0130
:102840002E1B3F0B2F3F3F4798F52091400222233C
:10285000B1F01092400220913E0230913F02821B63
:10286000930B8F3F9F4758F4205D3A4830933F02C7
:1028700020933E0280914F02886080934F028090A7
:102880004B0290904C020E0F1F1F109348020093B2
:10289000470287E492E0F701099580914B029091FD
:1028A0004C02892B29F4892819F081E08093400299
:1028B00080914502E82FEE0FEE0FE09345028FB1B5
:1028C00085FB662460F8712C7E9903C080E090E05F
:1028D00002C082E090E0862997298E2B80934502E2
:1028E000109144028F70E82FF0E0E756FE4F908180
:1028F00080914302890F8093430284306CF0E12F72
:10290000F0E0EF5BFD4F80818F5F808360E0812F7F
:102910000E947A0321E001C020E0809143028D3FB4
:1029200064F4E12FF0E0EF5BFD4F80818150808304
:1029300061E0812F0E947A0321E080914302082EFA
:10294000000C990B64E070E00E948D2A8093430292
:1029500021110E94DD0D0E94CF1990914602891726
:1029600009F44BCE8093460248CE59BC19BD09B438
:1029700000FEFDCF8091D8008F7D8093D80080919C
:10298000E00082608093E0008091E00081FDFCCF58
:102990000E94522438CEAF92BF92CF92DF92EF9234
:1029A000FF920F931F93CF93DF937C015B016A012A
:1029B000809110028A3018F001E010E002C00AE0B5
:1029C00010E0C1E0D0E0F894B501C701F601099527
:1029D0007894811115C021960C171D0794F0CC9F97
:1029E0009001CD9F300D300D112480E090E045E343
:1029F0004A95F1F70000019682179307C1F7E3CFDC
:102A000081E0DF91CF911F910F91FF90EF90DF90C8
:102A1000CF90BF90AF900895089508950895809144
:102A20009C02089580939702709399026093980294
:102A30008091A702843001F582E08093E9008FEF56
:102A40009091E800815095FD06C095ED9A95F1F7BB
:102A500000008111F5CF8091E80085FF0DC040E0B6
:102A600050E063E070E087E992E00E94D91B80911A
:102A7000E8008E778093E8000895BC0184E00C9410
:102A80001215BC0183E00C941215CF93DF9321E063
:102A90002093E9002FEF3091E800215035FD06C06A
:102AA00035ED3A95F1F700002111F5CF2091E800BE
:102AB00025FF14C0EC0140E050E068E070E00E94A7
:102AC000D91B8091E8008E778093E80088E0FE01B2
:102AD000ADE9B2E001900D928A95E1F7DF91CF91D7
:102AE00008950F931F93CF93DF93EC0100E010E064
:102AF00080915701282F30E00217130724F5909199
:102B000055019801290F311DA901440F551F240FAC
:102B1000351F2D5A3D4F869590E04C8108171907B7
:102B20001CF4442331F002C0411103C040918602DD
:102B300001C040E060918502809184020E94852559
:102B40000F5F1F4FD5CF0E9485248C8190E00196A6
:102B5000817099278C83DF91CF911F910F910895F8
:102B60008F929F92AF92BF92CF92DF92EF92FF929D
:102B70000F931F93CF93DF938C01FC014481C42FEB
:102B8000D0E09E01DE010E94D12A9B01AC010E948F
:102B9000E72A6B017C01E0E2F0E0EC1BFD0BA5E510
:102BA000B0E09B01AC010E94E72A4B015C019F0150
:102BB000DF010E94C92A9B01AC010E94F22A9B01FD
:102BC000AC012C0D3D1D4E1D5F1DC501B4010E94C1
:102BD000A12AC22FD22F2A3228F4F3E02F9F90018E
:102BE00011240DC025E530E02C1B3109C901880FE7
:102BF000991F280F391F37FF02C02F5F3F4F3595B0
:102C00002795C22FC095F12C85E5E82EED1A80910D
:102C10005701F816C8F4F1FC02C08E2D01C08D2FAB
:102C2000909155012F2D30E0290F311DA901440F3E
:102C3000551F240F351F2D5A3D4F4C2F6091850293
:102C40000E948525F394E3CF0E948524F8018481B6
:102C5000811102C091E003C0803219F49FEF90937C
:102C6000520190915201890FF8018483DF91CF9135
:102C70001F910F91FF90EF90DF90CF90BF90AF909A
:102C80009F908F9008951F93CF93DF93EC018C81D9
:102C9000811109C081E08C831092510292E09093DF
:102CA00051018093500180915501909156018917EF
:102CB00070F4E82FF0E09F01220F331FE20FF31FA3
:102CC000ED5AFD4F1182108212828F5FF0CF10E01B
:102CD000609157011617C0F5E12FF0E070E0CF01C9
:102CE0000E948D2A20915501820F20915102022EBF
:102CF000000C330B90E0E217F307CCF02091510168
:102D0000022E000C330B2E173F078CF09C01220F74
:102D1000331F820F931F9C012D5A3D4F4091860215
:102D200060918502809184020E9485250BC0FC0180
:102D3000EE0FFF1F8E0F9F1FFC01ED5AFD4F1182FA
:102D4000108212821F5FC4CF0E948524809150019F
:102D500020915102280F2093510290915101980F18
:102D60009093510119165CF4022E000C330B409124
:102D7000570150E0415051092417350734F081952F
:102D800080935001813009F41C82DF91CF911F9113
:102D900008958F929F92AF92BF92CF92DF92EF925F
:102DA000FF920F931F93CF93DF93EC018A8180FFF3
:102DB00003C0BB24BA9402C0BB24B3948C8181119C
:102DC0000DC081E0B81206C08091570181508093F8
:102DD000500202C01092500281E08C83A12C90908E
:102DE0005701A91408F03EC080915501CA2CD12C7E
:102DF0008601080F111DC801880F991F080F191FA0
:102E00000D5A1D4FF80111821082128234E0E32E18
:102E1000F12C812C80915002880D813114F08F703B
:102E200002C087FD890D082E000C990BC816D90623
:102E300091F4809186028E9DA0018F9D500D1124EA
:102E400055954795559547959801609185028091D4
:102E500084020E9485258B0CF1E0EF1AF108D1F66F
:102E6000A394BDCF0E9485248091500291E0B912B5
:102E70000EC0811107C0809157018150809350028C
:102E80001C820FC0815080935002BC820AC090E027
:102E900001966091570170E00E948D2A8093500244
:102EA0008C83DF91CF911F910F91FF90EF90DF9076
:102EB000CF90BF90AF909F908F900895FF920F9307
:102EC0001F93CF93DF93EC01F12C0FEF10E0609193
:102ED0005701F616F0F4809155012F2D30E0280FA0
:102EE000311DC901880F991F280F391F2D5A3D4FD9
:102EF00070E0C8010E948D2A962F8C814091860235
:102F000060918502F99E800D11240E948525F3941D
:102F1000DECF0E9485249A818C8190FF02C08F5F52
:102F200001C081508C83DF91CF911F910F91FF9051
:102F300008950F931F93CF93DF9300D01F92CDB7C7
:102F4000DEB78C018091520281110AC09E012F5F71
:102F50003F4F4FEF6FEF0E9485258A818093520289
:102F6000F8018481813051F028F0823061F4409181
:102F700052020AC08091520240E007C060915202A2
:102F800040E080E003C040E080E060E00E940C256B
:102F9000F801848190E0019663E070E00E948D2A40
:102FA00084830F900F900F90DF91CF911F910F911D
:102FB0000895CF93DF93EC01E3E8F2E0438162816F
:102FC0008C810E941B268C818F5F8C83DF91CF9137
:102FD0000895CF93DF93EC01EC81F0E0E651FF4FD1
:102FE0004491E3E8F2E0628181810E941B268C819A
:102FF0008F5F8C83DF91CF9108952091E400309111
:10300000E50095E64091EC00842F817040FF23C0DD
:103010008091E80080FD1DC08091A702882399F06F
:10302000853099F08091EB0085FD11C04091E4005E
:103030005091E5002417350729F3915011F09A01BA
:10304000E1CF84E0089582E0089583E0089581E06F
:10305000089580E008954091E80042FFDDCF089593
:103060008091A90287FF11C08091E80082FD05C010
:103070008091A7028111F8CF11C08091E8008B7771
:103080000BC08091A702882349F08091E80080FF5F
:10309000F8CF8091E8008E778093E8000895982F0C
:1030A000973068F59093E900981739F07091EC002B
:1030B0002091ED005091F00003C0242F762F50E0B6
:1030C00021FD02C09F5FECCF3091EB003E7F30933B
:1030D000EB003091ED003D7F3093ED003091EB003F
:1030E00031603093EB007093EC002093ED0050932F
:1030F000F0002091EE0027FDE5CF80E008958F706D
:103100008093E90081E008952091AF023091B002F0
:103110002617370748F06115710539F42091E8004A
:103120002E772093E80001C0B901FC0120E0611571
:10313000710579F18091A7028823F1F18530F1F1D1
:103140008091E80083FD3CC08091E80082FD2EC0A4
:103150008091E80080FFEBCF2091F3008091F20096
:1031600090E0922B6115710551F08830910538F48B
:1031700021912093F100615071090196F3CF21E074
:10318000089709F020E08091E8008E778093E800AE
:10319000CECF2111CFCF0AC08091A702882361F042
:1031A000853061F08091E80083FD0AC08091E800DD
:1031B00082FFF2CF80E0089582E0089583E00895D1
:1031C00081E0089581E08093E00080E28093D80060
:1031D0001092C9008FE19EE40197F1F700C0000052
:1031E00087E090EBDC0180932D0390932E03A09356
:1031F0002F03B09330039CE088E10FB6F894A895B4
:10320000809360000FBE90936000FFCF78941F9270
:103210000F920FB60F9211248F939F93AF93BF938A
:103220008091930290919402A0919502B0919602A0
:103230000196A11DB11D8093930290939402A093D7
:103240009502B0939602BF91AF919F918F910F908D
:103250000FBE0F901F9018959C014FB7F894809166
:10326000930290919402A0919502B09196024FBF63
:10327000821B930B08952FB7F8946091930270917D
:10328000940280919502909196022FBF08952FB7D6
:10329000F8948091930290919402A0919502B0913C
:1032A00096022FBF08951F920F920FB60F9211240E
:1032B0008F939F93AF93BF9380919202811113C01C
:1032C0008091930290919402A0919502B091960200
:1032D0004196A11DB11D8093930290939402A093F7
:1032E0009502B0939602BF91AF919F918F910F90ED
:1032F0000FBE0F901F9018959C012A5F3F4FFC0155
:103300004281461301C01282019682179307B9F7D2
:1033100008959C01FC0132969FEF80E04191461791
:1033200089F09F3F19F4411101C0982F8F5F8630BB
:10333000A9F79F3F39F0F901E90FF11D97FDFA95C3
:103340006283089508952091900230919102281788
:10335000390771F09093910280939002E0918E0270
:10336000F0918F02309721F00084F185E02D0994CF
:10337000089520918C0230918D022817390771F041
:1033800090938D0280938C02E0918E02F0918F02D7
:10339000309721F00680F781E02D099408950E946E
:1033A000F60B882351F0E0918E02F0918F02309756
:1033B00021F00190F081E02D099480E008950F93B1
:1033C0001F93CF93DF93C42FD22FFC0182818823D8
:1033D000C9F040938B020E94471990938A02809310
:1033E000890280E28C0F883008F072C0C77081E0DB
:1033F00001C0880FCA95EAF7DF91CF911F910F9115
:103400000C94642480918B0248133DC08091890202
:1034100090918A020E942C19883C9105A0F510E237
:103420001D0FCD17E9F080E28C0F883040F4C77093
:1034300081E001C0880FCA95EAF70E945D24183028
:1034400090F581E09D2F977001C0880F9A95EAF75B
:103450000E946424093369F560E570E089E32CC0BB
:10346000093319F460E570E002C060E070E0802F7D
:103470000E946E24183060F5D77081E001C0880F7B
:10348000DA95EAF70AC080E28C0F883008F5C77039
:1034900081E001C0880FCA95EAF7DF91CF911F91B3
:1034A0000F910C945D24093351F460E570E089E3D9
:1034B00009C060E070E0802F0E946E24DDCF60E0E4
:1034C00070E0802FDF91CF911F910F910C946E24AB
:1034D000DF91CF911F910F910895FC01680F791F23
:1034E0008FEF91E3E617F70771F02191822728E02B
:1034F00030E087FF03C0880F892701C0880F215063
:103500003109B9F7EFCF08958F929F92AF92BF9292
:10351000CF92DF92EF92FF920F931F93CF93DF939F
:10352000843048F4811108C0909180009F77909377
:1035300080002D9806C083E0909180009068909361
:103540008000A0918600B0918700282F30E00E9473
:10355000D12A23E030E040E050E00E94A12A002779
:10356000122F232F342F012F122F232F3327809137
:103570008600909187006CE070E00E94792A6017C5
:10358000710730F0C80169E070E00E94792A5EC0DE
:103590008091860090918700E0908600F0908700EF
:1035A000E0918600F0918700C6E0D0E0BE010E9465
:1035B000792A060F171F211D311D4801590185E089
:1035C000880C991CAA1CBB1C8A95D1F7C701BE01A7
:1035D0000E94792A6F01E12CF12CA7019601260F98
:1035E000371F411D511DC501B4010E94A12A690167
:1035F0007A01E0918600F0918700CA01B9010E942A
:10360000692A9B01AC01DF010E94E72A9B01AC0102
:10361000C701B6010E94692ADC01CB012FE0B695F3
:10362000A795979587952A95D1F7009186001091D7
:10363000870020E030E0081719072A073B0728F425
:103640006091860070918700CB01BC017093890066
:1036500060938800DF91CF911F910F91FF90EF90C1
:10366000DF90CF90BF90AF909F908F900895682F7C
:1036700086E090E00C94352A843008F083E0909145
:1036800088029770282F220F220F220F922B9093DF
:103690008802987F21E009F420E09091880220FBC5
:1036A00090F9909388020E94841A809188020C9469
:1036B000371B8091880280FD13C08160809388024F
:1036C000813019F489E080938802809188020E94F9
:1036D000371B809188028695869586950C94841A6E
:1036E000089580E090E00E942F2A893E9E4F51F07D
:1036F0000E94460E809188028470896180938802BE
:103700000E94371B86E090E00E94212A8093880265
:10371000282F26952695269530E02430310524F073
:1037200087708861809388028091880280FF04C03E
:1037300086958695869501C080E00C94841A9091B8
:10374000830290FF04C09695981740F003C0811142
:1037500005C090E0961710F40C94622761E00C9479
:103760001927882311F0FA0101C0FB010994EDE447
:10377000F2E01182828184608283089560918302E5
:10378000669570E04BE050E085E491E00E94FA2AF3
:10379000892B19F481E080934E020E944B0C909388
:1037A00048028093470280914F02846080934F02C9
:1037B0000895EF92FF920F931F93CF93DF937C01B5
:1037C0008B010E94FD17811119C0E7010115110538
:1037D000A1F08091E80085FD0AC08091E8008E7715
:1037E0008093E8000E94FD17882381F307C0899128
:1037F0008093F10001501109E9CF80E0DF91CF9172
:103800001F910F91FF90EF9008951F93CF93DF9337
:10381000CDB7DEB7AA970FB6F894DEBF0FBECDBF07
:10382000E9EAF2E081EB92E02091F10021938E171A
:103830009F07D1F78091AA02833009F461C030F468
:10384000813071F0823009F49BC0B2C08A3009F433
:1038500087C08B3009F46CC0893009F0A9C020C042
:103860008091A902813A09F0A3C08091E800877F86
:103870008093E8008091AD029091AE02892B21F4F3
:1038800068E08DE992E003C060E080E090E070E0E5
:103890000E9484188091E8008B778093E80088C0AC
:1038A0008091A902813209F083C08091AD0290918C
:1038B000AE02029708F07CC08091E800877F809379
:1038C000E8008091E80082FD05C08091A702811187
:1038D000F8CF6EC02091F3008091F20090E0922B1F
:1038E000029731F48091F100813011F0863021F49B
:1038F0008091F10080939C028091E8008B7754C006
:103900008091A902813A09F053C08091AD02909153
:10391000AE02892B09F04CC08091E800877F80932C
:10392000E8008091E80080FFFCCF8091580137C00B
:103930008091A9028132E1F58091AD029091AE02B1
:10394000892BB1F58091E800877F8093E8000E9481
:1039500030188091AB02809358010E94522428C0F5
:103960008091A902813221F58091E800877F8093C0
:10397000E8000E9430188091AC0280939B0218C02E
:103980008091A902813AA1F48091E800877F809319
:10399000E8008091E80080FFFCCF80919B0280933B
:1039A000F1008091E8008E778093E8000E94301843
:1039B0008091E80083FFCEC18091A9029091AA0274
:1039C000492F50E04A30510508F0C4C1FA01EE59C0
:1039D000FF4F0C94C32A803821F0823809F0BAC115
:1039E00008C08091A5029091A602992389F0826077
:1039F0000FC08091AD028F70873008F0ABC180930B
:103A0000E9008091EB0085FB882780F91092E9009E
:103A10009091E800977F9093E8008093F1001092D6
:103A2000F10065C1282F2D7F09F094C1882319F07A
:103A3000823061F08FC18091AB02813009F08AC180
:103A4000933009F080E08093A6022EC08091AB02F3
:103A500081112AC08091AD028F702FEF280F263080
:103A600008F078C18093E9002091EB0020FF1CC092
:103A7000933021F48091EB00806214C09091EB00B0
:103A800090619093EB0021E030E0A90102C0440F67
:103A9000551F8A95E2F74093EA001092EA00809160
:103AA000EB0088608093EB001092E9008091E800C1
:103AB000877F20C181114EC11091AB021F77809189
:103AC000E3008078812B8093E3008091E800877F7A
:103AD0008093E8000E9430188091E80080FFFCCFBE
:103AE0008091E30080688093E300111102C082E0BE
:103AF00001C083E08093A7022DC18058823008F076
:103B000029C18091AB029091AC028C3D53E09507A6
:103B100079F583E08A838AE289834FB7F894DE01DE
:103B2000139620E03EE051E2E32FF0E0509357007F
:103B3000E49120FF03C0E295EF703F5FEF708E2F9E
:103B400090E0EA3010F0C79601C0C0968D939D9327
:103B50002F5F243149F74FBF8091E800877F809322
:103B6000E8006AE270E0CE0101960E948418AEC0BF
:103B70004091AD025091AE02292F332723303105F9
:103B8000A9F068F42130310509F4F3C02230310581
:103B900009F0E0C08BE390E0ECE5F2E044C02132B4
:103BA000310521F12232310571F1D4C099278130DC
:103BB0009105A1F058F0029709F0CCC0E9EAF2E0D3
:103BC000E4918E2F90E0E9EAF2E02AC0E7EDF2E01E
:103BD000E4918E2F90E0E7EDF2E022C0E7ECF2E016
:103BE000E4918E2F90E0E7ECF2E01AC04115510508
:103BF00009F4C4C04130510509F0ACC089E090E03F
:103C0000E7E8F2E010C04115510509F4BCC04130AD
:103C1000510509F09FC082E390E0EAEEF1E003C0B5
:103C2000009709F497C02091E800277F2093E800CF
:103C30002091AF023091B0028217930708F49C01E3
:103C400040E02115310589F18091A702882309F40C
:103C50003DC08530D9F18091E80083FD37C0809167
:103C6000E80082FD2FC08091E80080FFEACF4091FC
:103C7000F3008091F20090E0942B2115310559F06A
:103C80008830910540F444914093F10031962150E1
:103C900031090196F2CF41E0089709F040E08091A8
:103CA000E8008E778093E800CCCF4111CDCF0AC0D9
:103CB0008091A702882351F0853041F08091E8007F
:103CC00083FD04C08091E80082FFF2CF8091E8007C
:103CD0008B778093E8003EC08038E1F58091E80062
:103CE000877F8093E8008091A8028093F100809103
:103CF000E8008E778093E8000E9430182BC0811175
:103D000029C08091AB029091AC029927029714F5DB
:103D10008091E800877F8093E8001091AB021093B8
:103D2000A8020E943018111106C08091E30087FD9F
:103D300002C081E001C084E08093A70242E061EC10
:103D400081E00E944F1842E261EC82E00E944F182D
:103D50008091A7028091E80083FF1AC08091E8005B
:103D6000877F8093E8008091EB0080628093EB0076
:103D70000FC082E190E0E7E9F2E055CF89E090E002
:103D8000EEE6F2E050CF80E490E0ECE1F2E04BCFE1
:103D9000AA960FB6F894DEBF0FBECDBFDF91CF91CC
:103DA0001F9108951F920F920FB60F9211242F9317
:103DB0003F934F935F936F937F938F939F93AF93B3
:103DC000BF93CF93DF93EF93FF93C091E900CF7040
:103DD0008091EC00D82FD17080FDD0E81092E900DE
:103DE0008091F000877F8093F00078940E94051CFA
:103DF0001092E9008091F00088608093F000CD2B54
:103E0000CF70C093E900FF91EF91DF91CF91BF9107
:103E1000AF919F918F917F916F915F914F913F9162
:103E20002F910F900FBE0F901F901895E8EDF0E0C6
:103E300080818E7F80831092E2001092DA001092CF
:103E4000E100A0EEB0E08C9181608C9380818F774F
:103E5000808319BCA7EDB0E08C918E7F8C9380811C
:103E60008F7E808310929A020895CF92DF92EF9214
:103E7000FF920F931F93CF93DF93C8EDD0E088811B
:103E80008F7E8883E7EDF0E080818160808384E02D
:103E900082BF81E080939A0288818E7F888302EEC0
:103EA00010E0F80110821092DA0081EEC82ED12CB9
:103EB000F601108288818F77888388818068888363
:103EC00088818F7D888319BC1092A7021092A80266
:103ED0001092A6021092A50290EEE92EF12CF701A5
:103EE00080818B7F808388818160888342E060E06D
:103EF00080E00E944F18F60180818E7F8083F80158
:103F0000808181608083808188608083F7018081E7
:103F10008E7F8083888180618883DF91CF911F911C
:103F20000F91FF90EF90DF90CF9008951F920F9226
:103F30000FB60F9211242F933F934F935F936F937C
:103F40007F938F939F93AF93BF93EF93FF93809152
:103F5000E10082FF09C08091E20082FF05C08091EC
:103F6000E1008B7F8093E1008091DA0080FF2AC01E
:103F70008091D80080FF26C08091DA008E7F8093E8
:103F8000DA008091D90080FF18C080E189BD82E10C
:103F900089BD09B400FEFDCF81E08093A702809126
:103FA0009A0281110FC00E94161F0E94351F809136
:103FB000E20084608093E20005C019BC1092A70261
:103FC00010929A028091E10080FF17C08091E20078
:103FD00080FF13C08091E2008E7F8093E200809189
:103FE000E20080618093E2008091D800806280933B
:103FF000D80019BC85E08093A7028091E10084FF7E
:1040000030C08091E20084FF2CC080E189BD82E154
:1040100089BD09B400FEFDCF8091D8008F7D8093CB
:10402000D8008091E1008F7E8093E1008091E200D2
:104030008F7E8093E2008091E20081608093E200B5
:104040008091A802882311F084E007C08091E300EA
:1040500087FD02C081E001C083E08093A7028091C8
:10406000A7028091E10083FF27C08091E20083FFD7
:1040700023C08091E100877F8093E10082E08093FC
:10408000A7021092A8028091E1008E7F8093E10048
:104090008091E2008E7F8093E2008091E200806157
:1040A0008093E20042E060E080E00E944F1880913F
:1040B000F00088608093F000FF91EF91BF91AF9185
:1040C0009F918F917F916F915F914F913F912F9130
:1040D0000F900FBE0F901F9018959091D101809175
:1040E0002C03982B9093B1028091D201882389F000
:1040F000892B8093B102E3EBF2E097E080E09150EE
:1041000029F021912223D9F38F5FF9CF81110E94E9
:10411000B60E48E050E064E273E081EB92E00E946A
:10412000072B892BA9F088E0E1EBF2E0A4E2B3E0F1
:1041300001900D928A95E1F7E0918E02F0918F0245
:10414000309731F00280F381E02D81EB92E0099409
:10415000089580E090E00E94B91980E090E00E940C
:10416000A31910922C030C946D208091220390913E
:10417000F102891719F08F5F8770FBCF08950F93B5
:104180001F93CF93DF938091F00282958F7009F097
:104190005DC08091ED02882309F458C0809122030C
:1041A0001091F1026091EB027091EC02C091EE026D
:1041B000D091EF0291E06F3F09F090E0292F06E0E7
:1041C000811709F443C0209721F07F3F21F030E0B0
:1041D00003C031E001C0322F90E030FD34C0089FB1
:1041E000F001099FF00D1124DF01AE50BD4F119673
:1041F0003C911197371327C03C91361324C0129677
:104200003C91129731111FC013964D915C911497F8
:104210004C1B5D0B483C5105B0F48091F0028F704F
:1042200080618093F002E950FD4F80818F70806142
:1042300080838BEE92E00E949503DF91CF911F91D6
:104240000F910C94B52001968770BACFDF91CF9172
:104250001F910F9108958F929F92AF92BF92DF921C
:10426000EF92FF920F931F93CF93DF9380902102E1
:1042700090902202A0902302B09024024091D3019A
:104280005091D4016091D5017091D601842A952A6C
:10429000A62AB72ACFE1D0E02AE0D22EE92EF12CCF
:1042A000082F10E0D501C4010C2E04C0B695A795C7
:1042B000979587950A94D2F780FD04C0219790F7CF
:1042C00080E019C0DC9EF001DD9EF00D1124EE0DA2
:1042D000FF1D83E0EE0FFF1F8A95E1F7E00FF11F4E
:1042E000EE0FFF1FE552FD4F859194910E94540CF3
:1042F000019721F38C2FDF91CF911F910F91FF90A8
:10430000EF90DF90BF90AF909F908F900895CF93E4
:10431000DF93D82FC92F0E942B21EC2FF0E09AE0D9
:10432000899FE00DF11D112483E0EE0FFF1F8A9598
:10433000E1F7ED0FF11DEE0FFF1FE552FD4F8591E7
:1043400094910E94540CDF91CF910895FC018081DB
:1043500091810E94872192959F70963079F010F498
:10436000925001C09A50923068F4803F69F018F47E
:10437000883E40F409C0843F29F406C0883E20F0FE
:10438000813F11F080E0089581E008959F92AF92FF
:10439000BF92CF92DF92EF92FF920F931F93CF9332
:1043A000DF93CDB7DEB761970FB6F894DEBF0FBECF
:1043B000CDBF8C0185E0F801DE011D9601900D92C4
:1043C0008A95E1F7F801E2809091EB026091EC02AE
:1043D0004091EE025091EF024115510531F06F3FCF
:1043E00031F481E09F3F19F403C081E001C080E017
:1043F000F82FF1709F2E80FD1AC1F80130812181C4
:10440000C380D4808BEEA82E82E0B82EF090ED020F
:10441000F601E41BF50BFF2009F4C6C08091F00201
:10442000E83CF10508F091C0482F407F09F050C0EA
:10443000621311C093130FC0FE2CE1100CC08F70DB
:1044400080618093F002C5010E9495038091F00283
:10445000F801858329C1CD2831F02F3F31F481E067
:104460003F3F19F403C081E001C080E080FD03C03C
:1044700081E08E2502C080E090E0F82FF170FF2EE1
:1044800080FF1CC0809122034091F10256E0841706
:1044900009F4E8C090E0589FF001599FF00D1124F5
:1044A000EE50FD4F6181261306C06081631303C087
:1044B0006281E61203C001968770E9CFFE2CEE20E0
:1044C00009F4F2C08091F00281608093F00249C04B
:1044D000621306C0931304C0E11002C0F80186C045
:1044E000C8010E94A621882351F1EE2041F12091BC
:1044F000F002822F82958F7090E0029774F0809185
:10450000EB029091EC0298878F831986DB86CA862E
:104510002C87CE0107960E94950386E0F801ABEE4A
:10452000B2E001900D928A95E1F70E94BF200AC087
:104530006217C9F0C8010E94A62181111EC0C801DE
:104540000E949503FF24F394AFC0482F407F81F76A
:104550008BEE92E00E94950386E0F50111928A9518
:10456000E9F7F12CA1C09313E5CFE110E3CFF801F7
:104570008583C8010E94950354C0EE2001F3209169
:10458000F002822F82958F7090E0029734F2809132
:10459000EB029091EC029A8389831B82DD82CC82AC
:1045A0002E83CE010196B7CFE83CF105D0F5FE2C65
:1045B000EE2029F2621327C0931325C02091F00248
:1045C00020FD18C0822F82958F70482F50E0411532
:1045D000510581F0F80125834F30510541F08F5F7F
:1045E000982F9295907F822F8F70892B8583C80199
:1045F0000E94950386E0F801ABEEB2E001900D92C7
:104600008A95E1F751C0C8010E94A621811185CF8A
:104610008091F00281608093F002C8010E949503AE
:1046200043C086E0F50111928A95E9F73DC0EE207E
:1046300009F485CFC8010E94A621F82E882309F429
:104640007ECF86E0F801ABEEB2E001900D928A9544
:10465000E1F78091EB029091EC020E9487210E9489
:10466000BF2022C03D872E878D859E850E94872191
:10467000292F22952F70223028F49F7039F0811154
:1046800005C00BC0243028F49F7049F4805E883048
:1046900020F0C8010E9495039F2CF92C05C0F80159
:1046A0009581907F99F7F9CF8F2D61960FB6F89489
:1046B000DEBF0FBECDBFDF91CF911F910F91FF9055
:1046C000EF90DF90CF90BF90AF909F90089528E03B
:1046D000929F800D1124682F669566956695982F98
:1046E000977085E0689FB001112440E050E080E0C1
:1046F000FB01E40FF51FE754FD4F208130E0092E48
:1047000002C0369527950A94E2F721703327042ECC
:1047100001C0220F0A94EAF7822B4F5F5F4F4530AA
:10472000510531F7089528E0929F800D1124E82F5C
:10473000E695E695E695877051E001C0550F8A959C
:10474000EAF785E0E89FF0011124E754FD4F20E0EF
:1047500030E070E04081CB01022E02C09695879533
:104760000A94E2F7817081958427852384278193B9
:104770002F5F3F4F2530310569F70895609321027F
:104780007093220280932302909324020C94A92018
:104790000F931F9341E050E060E070E004C0440FCD
:1047A000551F661F771F8A95D2F7409550956095E3
:1047B00070958091210290912202A0912302B091E4
:1047C00024028A019B01082319232A233B23C901C0
:1047D000B8011F910F910C94BE2320912303809563
:1047E000822380932303982F977099F430E0482F09
:1047F000082E000C550B2417350759F0909126020E
:1048000092FD07C08595859585950E94C8231092D5
:1048100023030895CF93C0912602C2FB992790F9F4
:10482000981799F080FBC2F9C09326026091250287
:1048300084E090E00E94352A6C2F82E290E00E9492
:10484000352A82E0CF910C94ED23CF9108950F93F8
:104850001F9341E050E060E070E004C0440F551F3A
:10486000661F771F8A95D2F78091210290912202CC
:10487000A0912302B09124028A019B01082B192BDD
:104880002A2B3B2BC901B8011F910F910C94BE2319
:104890006093D3017093D4018093D5019093D60196
:1048A0000C94A9201092D10186E0E3EBF2E0DF0145
:1048B0001D928A95E9F70C94A920882321F00E9483
:1048C000BC0E0C946D200895882339F09091D1018D
:1048D000892B8093D1010C946D2008951F93CF9361
:1048E000DF93182FEB010E94C327209741F08FE937
:1048F0009FE00197F1F700C000002197F6CF812FCC
:10490000DF91CF911F910C946C27CF92DF92EF92A1
:104910000F931F93CF93DF93CDB7DEB7E0970FB61A
:10492000F894DEBF0FBECDBF609154018091830229
:1049300080FF0AC0E0E2F5E0AE014F5F5F4F8E01FD
:104940000F5C1F4FCA0114C0809155019091560110
:10495000891780F7E82FF0E09F01220F331FE20F45
:10496000F31FED5AFD4F1182108212828F5FF0CF3C
:10497000249130E0D901AA0FBB1F2A0F3B1FD90198
:10498000AD5ABD4FCD90DD90EC90DA01CD92DD9225
:10499000ED92AD013196A017B10751F72091530167
:1049A000FC01B3E02B9FE00DF11D11246E9A8EB136
:1049B0008F7B9EB190642FB7F894AF0133E0639F73
:1049C000400D511D1124E417F50789F0319168E07D
:1049D0009EB9000000C037FF8EB9330F000000C041
:1049E00000C000C08EB900C06A9591F7ECCF2FBF10
:1049F0008FE594E00197F1F700C00000E0960FB654
:104A0000F894DEBF0FBECDBFDF91CF911F910F9104
:104A1000EF90DF90CF9008959091830290FF16C0A1
:104A20009091550120915601921770F4E92FF0E012
:104A3000DF01AA0FBB1FEA0FFB1FED5AFD4F818359
:104A4000608342839F5FF0CF0C948524089580910A
:104A50008302282F269530E02115310519F4817045
:104A6000826005C02532310524F08170886480930E
:104A700083020895CF92DF92EF92FF926B017C0147
:104A80000E942725B701A60188E090E0FF90EF90F3
:104A9000DF90CF900C94472A80918702882319F0E9
:104AA000815080938702609183027091840280918B
:104AB0008502909186020C943A258091870283307A
:104AC00018F48F5F80938702609183027091840253
:104AD00080918502909186020C943A25E3E8F2E0F9
:104AE00087E1808311828FEF828383831482ADE418
:104AF000B2E012968C911297836012968C9360812B
:104B00007181828193810C943A25AF92BF92CF92AA
:104B1000DF92EF92FF920F931F93CF93DF93E82ED4
:104B2000F62EE901E42FF0E0611106C0E55EFB4FCF
:104B3000E4914E2F2E2F71C0062F10E0E55EFB4F43
:104B40004491F42FC42ED12C26E0829FC001112461
:104B50002FEF30E0B9010E94792A5BEA5603C001C9
:104B6000579F900D11248E0D911D8E0D911D582F64
:104B7000550F580FD901A01BB10BAC9DC001AD9DC5
:104B8000900DBC9D900D1124E92FF59ED0011124AC
:104B9000AB2FBB277901EA1AFB0AEC9CD001ED9CF4
:104BA000B00DFC9CB00D11245901A51AB108A09EAE
:104BB0007001A19EF00CB09EF00C1124EF2CFF248C
:104BC0002E193F092C9D80012D9D100D3C9D100D2F
:104BD0001124212F6230710591F048F4611571059F
:104BE000E1F061307105B9F4242F4B2F16C0643009
:104BF000710569F040F06630710579F00CC0242F22
:104C0000492FE12F0AC0492FEF2F2B2F06C0292F44
:104C1000E42F412F02C0292FEB2F49832883EA83F9
:104C2000DF91CF911F910F91FF90EF90DF90CF9088
:104C3000BF90AF900895CF93DF9300D01F92CDB770
:104C4000DEB79091830290FF0AC09E012F5F3F4F15
:104C50000E9485254B8169818A810E940C250F90D5
:104C60000F900F90DF91CF910895AF92BF92CF92A6
:104C7000DF92EF92FF920F931F93CF93DF9300D0B9
:104C80001F92CDB7DEB7182FF62E042FE22E90918B
:104C9000830290FF7EC0E92FE695AE2FB0E0A755C6
:104CA000BE4F8C9180934D029E7F923061F49E01A5
:104CB0002F5F3F4F812F0E9485254B8169818A811B
:104CC0000E940C2543C0823019F4009186023EC038
:104CD000863019F41091840239C08930D9F38931B2
:104CE000A9F5E9518E2F8170D82EE695F0E0E55EAA
:104CF000FA4FA590B490C12CBB2460915701C61601
:104D000018F52C2D30E0A29EC001A39E900DB29EFE
:104D1000900D112470E00E94792A812FD11002C0D9
:104D2000860F01C0861B90915501290F311DA901E5
:104D3000440F551F240F351F2D5A3D4F402F6F2D07
:104D40000E948525C394D9CF0E9485248091840236
:104D5000181308C080918502F81204C08091860261
:104D6000081729F080914F02826080934F021093C0
:104D70008402F092850200938602EE2051F0609149
:104D800083027091840280918502909186020E9434
:104D90003A250F900F900F90DF91CF911F910F91B7
:104DA000FF90EF90DF90CF90BF90AF900895E3E831
:104DB000F2E0438121E1421B08F440E021E06281FE
:104DC00081810C943526E3E8F2E0438121E1420F32
:104DD00008F44FEF21E0628181810C943526E3E8ED
:104DE000F2E0628121E1621B08F460E021E043818E
:104DF00081810C943526E3E8F2E0628121E1620FC3
:104E000008F46FEF21E0438181810C943526E3E8BB
:104E1000F2E0818121E04381628188500C94352643
:104E2000E3E8F2E0818121E043816281885F0C94B4
:104E300035269091830290FF3BC09170811102C092
:104E4000926006C0853210F0986402C0880F982BDB
:104E50009093830280914F02816080934F0266237A
:104E600051F060918302709184028091850290914B
:104E700086020E943A2560918302669570E04BE0BD
:104E800050E085E491E00E94FA2A892B19F00E94F3
:104E9000B71B02C00E94BE1B81E080934A0220E043
:104EA0004091860260918502809184020C9435269F
:104EB0000895809183028695815009F484E261E02F
:104EC0000C9419278091830286958F5F853208F0B4
:104ED00081E061E00C941927882309F453C0682FFE
:104EE000823869F40E94CF1981FF4CC069E381EBDD
:104EF00092E00E9489190E946D2069E30EC08338F8
:104F000091F40E94CF1980FF3DC063E581EB92E0F0
:104F10000E9489190E946D2063E581EB92E00E9456
:104F20007C190C946D20843869F40E94CF1982FF9B
:104F300029C067E481EB92E00E9489190E946D20EC
:104F400067E4EBCF8CEF860F813A38F380E2860F6F
:104F5000883048F4677081E001C0880F6A95EAF7ED
:104F60000E94BC0EDECF8BE5860F833020F480E0FC
:104F700090E00C94B919685A673120F480E090E011
:104F80000C94A3190895CF93882309F496C0C82FD1
:104F90008238B1F40E94CF1981FD8FC069E381EBA3
:104FA00092E00E9489190E946D202FEF81EE94E01B
:104FB000215080409040E1F700C0000069E317C035
:104FC0008338E1F40E94CF1980FD77C063E581EB5F
:104FD00092E00E9489190E946D202FEF81EE94E0EB
:104FE000215080409040E1F700C0000063E581EB74
:104FF00092E00E947C19CF910C946D208438B1F41A
:105000000E94CF1982FD59C067E481EB92E00E94B3
:1050100089190E946D202FEF81EE94E0215080408D
:105020009040E1F700C0000067E4E1CF8CEF8C0F07
:10503000813A80F4E3EBF2E089EB92E02191C21730
:10504000A1F18E179F07D1F76C2F81EB92E00E94A0
:105050008919D1CF80E28C0F883068F4C77081E065
:1050600090E001C0880FCA95EAF79091D101892B91
:105070008093D101C0CFEBE5EC0FE33040F4F0E0DA
:10508000E75AFE4F808190E0CF910C94B919C85A2D
:10509000C73198F4EC2FF0E0EE0FFF1FE45AFE4FFB
:1050A00080819181CF910C94A3196C2F81EB92E0B8
:1050B0000E947C190E946D20C7CFCF9108958EE188
:1050C000489B02C08150E1F7489BFECF0895589855
:1050D00080E28A95F1F7589A0895FC012AE02A9512
:1050E000F1F728E090E080E031E040E14A95F1F707
:1050F000880F489B02C08160932700C0000040E1F8
:105100004A95F1F7215089F720E12A95F1F729B165
:1051100000C0000030E13A95F1F72170922720811C
:10512000920F90830895EF92FF920F931F93CF9366
:10513000DF931F92CDB7DEB719828C017C01E60E9A
:10514000F11C0E151F0551F00E945F28CE0101963B
:105150000E946D28F80181938F01F3CF81E099813E
:10516000911180E00F90DF91CF911F910F91FF90EF
:10517000EF900895509A589A08955098589AE89A3E
:10518000E9E6F0E080818C7F80830895615091E0B2
:1051900001C0990F6A95EAF720E031E0992361F0A8
:1051A000492F482319F0589A232701C0589840E204
:1051B0004A95F1F79695F2CF222311F0589A01C043
:1051C000589880E28A95F1F758980895FF920F93C6
:1051D0001F93CF93DF93EC018C01060F111DC017B5
:1051E000D10741F0F9900E94672868E08F2D0E9456
:1051F000C628F5CFDF91CF911F910F91FF900895B1
:105200001F920F920FB60F9211240F931F932F939B
:105210003F934F935F936F937F938F939F93AF933E
:10522000BF93EF93FF93CF93DF931F92CDB7DEB77A
:1052300019820E945F28CE0101960E946D28082FD6
:10524000069506950695902F96959570202F2570BA
:10525000920F292F237096959695920F8770891338
:105260005FC0898181115CC0083008F059C080E1BD
:105270008A95F1F7589A509A82E08A95F1F700C022
:10528000589888E0089F80011124D801A050BF4F92
:105290001696ED91FC9117973097A9F060918A01CD
:1052A00070918B0114962D913C911597260F371F05
:1052B00011968D919C911297680F791F13964C91BE
:1052C00013978C910995F801E050FF4F6381662395
:1052D00051F080918A0190918B0124813581820F58
:1052E000931F0E94E6280E94672880E18A95F1F7C3
:1052F00058985098589A80E18A95F1F7F801E05053
:10530000FF4F6081662351F080918A0190918B015B
:1053100021813281820F931F0E9493280E945F286F
:105320000F90DF91CF91FF91EF91BF91AF919F913E
:105330008F917F916F915F914F913F912F911F912D
:105340000F910F900FBE0F901F9018950F931F9302
:10535000CF93DF93883091050CF06DC0EC01F89489
:10536000509A589885E08A95F1F700009C2F969501
:1053700095702C2F2570920F892F83709695969596
:1053800023E0CC0FDD1F2A95E1F7980F8E01092B42
:105390000E94672884E08A95F1F700C068E0802FBA
:1053A0000E94C62880E18A95F1F75098589A48994A
:1053B00002C000C0FCCF87E090E0489B08C0019786
:1053C00021F4509A589A789436C000C0F6CFFE0166
:1053D000E050FF4F6381662381F080918A019091B4
:1053E0008B0124813581820F931F0E9493288111A4
:1053F00004C0509A589A78941FC00E945F2880E297
:105400008A95F1F75898509A80E18A95F1F7C05043
:10541000DF4F6881662351F080918A0190918B0162
:1054200029813A81820F931F0E94E6280E946728F3
:10543000789481E001C080E0DF91CF911F910F91BE
:105440000895F999FECF92BD81BDF89A992780B54C
:105450000895A6E1B0E044E050E00C945B2AA8E196
:10546000B0E042E050E00C945B2A262FF999FECF81
:1054700092BD81BDF89A019700B4021639F01FBAA7
:1054800020BD0FB6F894FA9AF99A0FBE08950396C4
:10549000272F0E94362A0E94352A252F0E94362A5D
:1054A000242F0C94362A0196272F0E94362A0C941A
:1054B000352ADC01CB01FC01F999FECF06C0F2BD13
:1054C000E1BDF89A319600B40D9241505040B8F7C2
:1054D0000895DB018F939F930E94E72ABF91AF91BC
:1054E000A29F800D911DA39F900DB29F900D11243E
:1054F0000895AA1BBB1B51E107C0AA1FBB1FA6171B
:10550000B70710F0A61BB70B881F991F5A95A9F76C
:1055100080959095BC01CD01089597FB072E16F458
:10552000009407D077FD09D00E94792A07FC05D0A6
:105530003EF4909581959F4F0895709561957F4FAA
:105540000895A1E21A2EAA1BBB1BFD010DC0AA1FC4
:10555000BB1FEE1FFF1FA217B307E407F50720F0DC
:10556000A21BB30BE40BF50B661F771F881F991F57
:105570001A9469F760957095809590959B01AC01A0
:10558000BD01CF010895EE0FFF1F0590F491E02DAE
:1055900009940E94D12A332312F48A1B9B0B0C948A
:1055A000E22AA29FB001B39FC001A39F700D811D8D
:1055B0001124911DB29F700D811D1124911D08951C
:1055C0000E94D12AB7FF0895821B930B08950E9471
:1055D000D12AA59F900DB49F900DA49F800D911D81
:1055E00011240895B7FF0C94E72A0E94E72A821B32
:1055F000930B0895FC014150504030F00190061685
:10560000D1F73197CF010895882799270895FB0195
:10561000DC0104C08D910190801921F4415050406B
:10562000C8F7881B990B0895FB01DC0102C00190AB
:0E5630000D9241505040D8F70895F894FFCFE6
:10563E000000000100000000000000050100000055
:10564E00000000010600000000000001070000003D
:10565E000408000000000000010C00000000000023
:10566E00080D000000000000010F1545150E154134
:10567E00153D150C1501191A1B1C1D1E1F2021226C
:10568E00010201001000101001818283E200E90086
:10569E00EA00B500B600B700CD008301CC008A0148
:1056AE0092019401210223022402250226022702DE
:1056BE002A02B300B4006F007000EF01313267347C
:1056CE0097F4F1F0373392939500FF01000100003B
:1056DE00FFFF0000010001FF0000010202020206AE
:1056EE0006060909090909090F0F0F0F0F0F1515E6
:0E56FE00151819191919191919191919232430
:00000001FF
